:2000000012C02BC02AC029C028C027C026C025C024C023C022C021C020C01FC01EC01DC0B2
:200020001CC01BC01AC011241FBECFEDCDBF10E0A0E6B0E0E0E9F4E003C0C89531960D92AC
:20004000A036B107D1F710E0A0E6B0E001C01D92A136B107E1F7CFD11AC2D2CFCF93DF937C
:20006000CDB7DEB7E7E3F0E08FEF8083A1E3B0E0E1E3F0E0808188608C93A1E3B0E0E1E3C4
:20008000F0E0808184608C93E8E3F0E08FEF8083A2E3B0E0E2E3F0E0808188608C93A2E339
:2000A000B0E0E2E3F0E0808184608C9386E91ED080E358D082E31AD080E354D07ED180E3A7
:2000C00051D088E24FD0A7E3B0E0E7E3F0E0908180EF89238C938CE045D086E043D082E01B
:2000E00041D081E03FD0DF91CF910895CF93DF93CDB7DEB722970FB6F894DEBF0FBECDBF25
:200100008A838A81898304C058D189818150898389818823C9F722960FB6F894DEBF0FBEFF
:20012000CDBFDF91CF910895CF93DF93CDB7DEB721970FB6F894DEBF0FBECDBF88EC89835A
:2001400005C082E3D3DF89818150898389818823C1F721960FB6F894DEBF0FBECDBFDF9101
:20016000CF910895CF93DF93CDB7DEB721970FB6F894DEBF0FBECDBF898340E0698184E01C
:2001800023D08FE0B3DF21960FB6F894DEBF0FBECDBFDF91CF910895CF93DF93CDB7DEB713
:2001A00021970FB6F894DEBF0FBECDBF898340E0698180E009D021960FB6F894DEBF0FBE7F
:2001C000CDBFDF91CF910895CF93DF93CDB7DEB725970FB6F894DEBF0FBECDBF89836A833D
:2001E0004B838981282F33273D832C838C819D818330910554F42C813D8121303105DCF489
:200200008C819D810097E9F023C02C813D812330310571F08C819D818430910509F018C0C5
:20022000A2E3B0E0E2E3F0E08081877F8C9310C08B81805C8B838B81982F9F7780E8892B23
:2002400091DFA2E3B0E0E2E3F0E0808188608C93A2E3B0E0E2E3F0E0808184608C93A2E349
:20026000B0E0E2E3F0E0808184608C93A8E3B0E0E8E3F0E08081982F8FE0292F28239A81AA
:2002800080EF8923822B8C93A8E3B0E0E8E3F0E08081982F8FE0292F28239A8180EF8923B1
:2002A000822B8C93A2E3B0E0E2E3F0E080818B7F8C93A2E3B0E0E2E3F0E080818B7F8C93CA
:2002C0007CD0E7E3F0E08081803FE9F58A818295807F8A83A2E3B0E0E2E3F0E080818460DD
:2002E0008C93A2E3B0E0E2E3F0E0808184608C93A8E3B0E0E8E3F0E08081982F8FE0292FEC
:2003000028239A8180EF8923822B8C93A8E3B0E0E8E3F0E08081982F8FE0292F28239A81E5
:2003200080EF8923822B8C93A2E3B0E0E2E3F0E080818B7F8C93A2E3B0E0E2E3F0E0808157
:200340008B7F8C933AD025960FB6F894DEBF0FBECDBFDF91CF910895CF93DF93CDB7DEB70E
:2003600023970FB6F894DEBF0FBECDBF8B838B8199278330910509F003C080E48A8301C06B
:200380001A828A81898307C0498160E281E01CDF89818F5F89838981282F33278A819927F1
:2003A0000F962817390784F323960FB6F894DEBF0FBECDBFDF91CF910895CF93DF93CDB7DD
:2003C000DEB721970FB6F894DEBF0FBECDBF84E4898302C08981898189818150898389814E
:2003E0008F3FC1F721960FB6F894DEBF0FBECDBFDF91CF910895CF93DF93CDB7DEB72EDE13
:2004000080E2CADE80E2C8DE80E2C6DE80E2C4DE81E3C2DE83E3C0DE8AE3BEDE80E3BCDEB2
:2004200080E3BADE8AE3B8DE82E3B6DE83E3B4DE80E2B2DE80E2B0DE80E2AEDE80E2ACDE11
:2004400040E064E583E0C0DE89E4A6DE8DE4A4DE85E4A2DE82E5A0DE80E29EDE85E59CDEBE
:2004600088E69ADE82E798DE80E296DE87E594DE85E692DE83E690DE8BE68EDE85E68CDE9F
:1004800082E78ADE80E090E0DF91CF910895FFCF90
:00000001FF
